:1000000000308A001229000000000A108A100A112C
:10001000820720340C34013406340A108A100A1185
:100020008207303431343234333434343534363476
:100030003734383439344134423443344434453429
:1000400046340A108A100A1182075234653461342A
:10005000643479342E342E342E34003412080319CB
:100060003E2801308D008C018C0B34288D0B3328F9
:1000700027308C008C0B3A28920B312800340F303B
:10008000860519088C008C0EF0308C050C0886044F
:10009000000086150000861100348610F1306600DD
:1000A00006150000861500000608F0399900861133
:1000B0000000861506089800980E0F3098058611E6
:1000C00001306600190818048D000D089800981B6F
:1000D0004E2886109608031D8614000006110000A5
:1000E000861117089800980E0F3098051808990087
:1000F0003F2017080F399800180899003F20003456
:10010000FF308500E8306500F13086000130660080
:100110008E01643092002E200130900004301002D5
:1001200003189A28033099003F20053092002E20B2
:10013000900A8E28023099003F209001043010026E
:100140000318AB28100805209100960111089700AC
:100150004D20900A9E28162994010130120294071E
:100160001408803895009601150897004D2000343A
:1001700011088C000C300C020319D3280A300C0231
:100180000319DB280D300C020319DB2808300C02A0
:100190000319E1280E300C020319E6280F300C0277
:1001A0000319E828EA289601013097004D20023013
:1001B00092002E20F0280130920001309300AC20F4
:1001C000F0289601103097004D20F0280512F028F5
:1001D0000516F02801309600110897004D20F028F0
:1001E000003408308C000618F32890018C1706297B
:1001F0008C1306290310900C061890170C1706296B
:100200000C138C0BFA2810088D00112919308C1B47
:1002100006308D008D0B0A298C1BF8280C1B002939
:10022000FA28242984018301061480280C309100C7
:10023000B820900110082120003803192329900AC2
:100240009100B8201A29F1280D088F00851D2C294E
:100250000F089100B8204D290F088C008C0E0F302C
:100260008C050C080D20900010089100B8200F0894
:100270000F390D20900010089100B8202030910017
:10028000B8200E088E0A05300E02031D4D290130DC
:0E029000920001309300AC208E012329630000
:02400E00F93F78
:084000000E0006000300080099
:00000001FF
